 lcms

 Timestamp is 5356bb64 (Tue Apr 22 11:56:36 2014)

 Preferred load address is 10000000

 Start         Length     Name                   Class
 0001:00000000 0000fa08H .text                   CODE
 0002:00000000 000000b8H .idata$5                DATA
 0002:000000c0 000014a8H .rdata                  DATA
 0002:00001568 00000064H .rdata$debug            DATA
 0002:000015d0 00000004H .rdata$sxdata           DATA
 0002:000015d4 00000004H .rtc$IAA                DATA
 0002:000015d8 00000004H .rtc$IZZ                DATA
 0002:000015dc 00000004H .rtc$TAA                DATA
 0002:000015e0 00000004H .rtc$TZZ                DATA
 0002:000015e4 00000064H .idata$2                DATA
 0002:00001648 00000014H .idata$3                DATA
 0002:0000165c 000000b8H .idata$4                DATA
 0002:00001714 00000238H .idata$6                DATA
 0002:00001950 000002bdH .edata                  DATA
 0003:00000000 00000004H .CRT$XCA                DATA
 0003:00000004 00000004H .CRT$XCZ                DATA
 0003:00000008 00000004H .CRT$XIA                DATA
 0003:0000000c 00000004H .CRT$XIZ                DATA
 0003:00000010 000005f4H .data                   DATA
 0003:00000608 00002b08H .bss                    DATA
 0004:00000000 00000058H .rsrc$01                DATA
 0004:00000060 00000310H .rsrc$02                DATA

  Address         Publics by Value              Rva+Base     Lib:Object

 0000:00000000       __except_list              00000000     <absolute>
 0000:00000001       ___safe_se_handler_count   00000001     <absolute>
 0000:00009876       __ldused                   00009876     <absolute>
 0000:00009876       __fltused                  00009876     <absolute>
 0001:00000000       __cmsMalloc                10001000 f i cmscam02.obj
 0001:00000013       __cmsClampWord             10001013 f i cmscnvrt.obj
 0001:0000002c       _cmsD50_XYZ                1000102c f   cmscnvrt.obj
 0001:00000032       _cmsD50_xyY                10001032 f   cmscnvrt.obj
 0001:00000570       _cmsChooseCnvrt            10001570 f   cmscnvrt.obj
 0001:00000687       _cmsErrorAction            10001687 f   cmserr.obj
 0001:00000697       _cmsSetErrorHandler        10001697 f   cmserr.obj
 0001:000006a1       _cmsSignalError            100016a1 f   cmserr.obj
 0001:000007a4       __cmsCrc32OfGammaTable     100017a4 f   cmsgamma.obj
 0001:000007eb       _cmsAllocGamma             100017eb f   cmsgamma.obj
 0001:0000083d       _cmsFreeGamma              1000183d f   cmsgamma.obj
 0001:0000084b       _cmsFreeGammaTriple        1000184b f   cmsgamma.obj
 0001:00000876       _cmsDupGamma               10001876 f   cmsgamma.obj
 0001:000008a2       _cmsJoinGamma              100018a2 f   cmsgamma.obj
 0001:00000928       _cmsBuildParametricGamma   10001928 f   cmsgamma.obj
 0001:00000c8e       _cmsBuildGamma             10001c8e f   cmsgamma.obj
 0001:00000ca2       _cmsAllocSampledCurve      10001ca2 f   cmsgamma.obj
 0001:00000ced       _cmsFreeSampledCurve       10001ced f   cmsgamma.obj
 0001:00000d58       _cmsConvertSampledCurveToGamma 10001d58 f   cmsgamma.obj
 0001:00000dcd       _cmsConvertGammaToSampledCurve 10001dcd f   cmsgamma.obj
 0001:00000e58       _cmsReverseGamma           10001e58 f   cmsgamma.obj
 0001:00000ef0       __cmsEndPointsBySpace      10001ef0 f   cmsgmt.obj
 0001:00000fdf       __cmsWhiteBySpace          10001fdf f   cmsgmt.obj
 0001:0000100e       _Clamp_L                   1000200e f   cmsgmt.obj
 0001:00001029       _Clamp_ab                  10002029 f   cmsgmt.obj
 0001:00001046       _cmsDeltaE                 10002046 f   cmsgmt.obj
 0001:00001196       __cmsLCMScolorSpace        10002196 f   cmsgmt.obj
 0001:00001308       __cmsChannelsOf            10002308 f   cmsgmt.obj
 0001:000017fb       __cmsComputeGamutLUT       100027fb f   cmsgmt.obj
 0001:0000180e       __cmsPrecalculateGamutCheck 1000280e f   cmsgmt.obj
 0001:00001859       __cmsComputeSoftProofLUT   10002859 f   cmsgmt.obj
 0001:000019e9       __cmsComputePrelinearizationTablesFromXFORM 100029e9 f   cmsgmt.obj
 0001:00001cca       __cmsBuildKToneCurve       10002cca f   cmsgmt.obj
 0001:00001d38       _cmsCalcL16Params          10002d38 f   cmsintrp.obj
 0001:00001ddf       _cmsLinearInterpLUT16      10002ddf f   cmsintrp.obj
 0001:00001e7f       _cmsLinearInterpFixed      10002e7f f   cmsintrp.obj
 0001:00001edd       _cmsReverseLinearInterpLUT16 10002edd f   cmsintrp.obj
 0001:000020ec       _cmsTrilinearInterp16      100030ec f   cmsintrp.obj
 0001:00002329       _cmsTetrahedralInterp16    10003329 f   cmsintrp.obj
 0001:00002614       _cmsTetrahedralInterp8     10003614 f   cmsintrp.obj
 0001:00002c86       _cmsCalcCLUT16ParamsEx     10003c86 f   cmsintrp.obj
 0001:00002d56       _cmsCalcCLUT16Params       10003d56 f   cmsintrp.obj
 0001:00002f6f       __cmsCreateProfilePlaceholder 10003f6f f   cmsio0.obj
 0001:00002fad       __cmsSearchTag             10003fad f   cmsio0.obj
 0001:00002ff7       _cmsIsTag                  10003ff7 f   cmsio0.obj
 0001:00003013       __cmsInitTag               10004013 f   cmsio0.obj
 0001:000030bb       __cmsCreateProfileFromMemPlaceholder 100040bb f   cmsio0.obj
 0001:00003145       __cmsSetSaveToDisk         10004145 f   cmsio0.obj
 0001:0000319c       _cmsTakeMediaWhitePoint    1000419c f   cmsio0.obj
 0001:000031b7       _cmsTakeMediaBlackPoint    100041b7 f   cmsio0.obj
 0001:000031d2       _cmsTakeIluminant          100041d2 f   cmsio0.obj
 0001:000031ea       _cmsTakeRenderingIntent    100041ea f   cmsio0.obj
 0001:000031f2       _cmsSetRenderingIntent     100041f2 f   cmsio0.obj
 0001:000031fe       _cmsTakeHeaderFlags        100041fe f   cmsio0.obj
 0001:00003206       _cmsGetPCS                 10004206 f   cmsio0.obj
 0001:0000320e       _cmsSetPCS                 1000420e f   cmsio0.obj
 0001:0000321a       _cmsGetColorSpace          1000421a f   cmsio0.obj
 0001:00003222       _cmsSetColorSpace          10004222 f   cmsio0.obj
 0001:0000322e       _cmsGetDeviceClass         1000422e f   cmsio0.obj
 0001:00003236       _cmsGetProfileICCversion   10004236 f   cmsio0.obj
 0001:0000323e       _cmsSetDeviceClass         1000423e f   cmsio0.obj
 0001:00003271       __cmsAddLUTTag             10004271 f   cmsio0.obj
 0001:00003337       __cmsAddXYZTag             10004337 f   cmsio0.obj
 0001:00003351       __cmsAddTextTag            10004351 f   cmsio0.obj
 0001:00003375       __cmsAddGammaTag           10004375 f   cmsio0.obj
 0001:00003396       __cmsAddChromaticAdaptationTag 10004396 f   cmsio0.obj
 0001:00003396       __cmsAddChromaticityTag    10004396 f   cmsio0.obj
 0001:000033b0       __cmsAddSequenceDescriptionTag 100043b0 f   cmsio0.obj
 0001:000033d5       __cmsAddDateTimeTag        100043d5 f   cmsio0.obj
 0001:000033ef       __cmsAddNamedColorTag      100043ef f   cmsio0.obj
 0001:000033ef       __cmsAddColorantTableTag   100043ef f   cmsio0.obj
 0001:00003417       __cmsCalloc                10004417 f i cmsio1.obj
 0001:00004e81       _cmsReadICCLut             10005e81 f   cmsio1.obj
 0001:00005156       _cmsTakeColorants          10006156 f   cmsio1.obj
 0001:000051b2       _cmsReadICCMatrixRGB2XYZ   100061b2 f   cmsio1.obj
 0001:00005236       _cmsReadChromaticAdaptationMatrix 10006236 f   cmsio1.obj
 0001:00005292       _cmsReadICCGamma           10006292 f   cmsio1.obj
 0001:000052dd       _cmsReadICCGammaReversed   100062dd f   cmsio1.obj
 0001:0000537b       _cmsReadICCnamedColorList  1000637b f   cmsio1.obj
 0001:00005736       _cmsOpenProfileFromMem     10006736 f   cmsio1.obj
 0001:000069e8       _cmsAddTag                 100079e8 f   cmsio1.obj
 0001:00006c0b       __cmsSaveProfile           10007c0b f   cmsio1.obj
 0001:00006ccc       _cmsCloseProfile           10007ccc f   cmsio1.obj
 0001:00006d4b       _cmsAllocLUT               10007d4b f   cmslut.obj
 0001:00006d71       _cmsFreeLUT                10007d71 f   cmslut.obj
 0001:00006e58       _cmsDupLUT                 10007e58 f   cmslut.obj
 0001:00006f0a       __cmsValidateLUT           10007f0a f   cmslut.obj
 0001:00006f78       _cmsAlloc3DGrid            10007f78 f   cmslut.obj
 0001:00006ffc       _cmsAllocLinearTable       10007ffc f   cmslut.obj
 0001:00007264       _cmsSetMatrixLUT4          10008264 f   cmslut.obj
 0001:0000732f       _cmsEvalLUT                1000832f f   cmslut.obj
 0001:000078a3       __cmsBlessLUT8             100088a3 f   cmslut.obj
 0001:00007b42       _cmsEvalLUTreverse         10008b42 f   cmslut.obj
 0001:00007d8b       _cmsFreeMatShaper          10008d8b f   cmsmatsh.obj
 0001:000080ff       _cmsEvalMatShaper          100090ff f   cmsmatsh.obj
 0001:00008143       _cmsAllocMatShaper2        10009143 f   cmsmatsh.obj
 0001:000081ea       _cmsAllocMatShaper         100091ea f   cmsmatsh.obj
 0001:000082e2       _FixedMul                  100092e2 f   cmsmtrx.obj
 0001:000082f9       _FixedLERP                 100092f9 f   cmsmtrx.obj
 0001:0000831a       _VEC3init                  1000931a f   cmsmtrx.obj
 0001:00008333       _VEC3initF                 10009333 f   cmsmtrx.obj
 0001:00008379       _VEC3toFix                 10009379 f   cmsmtrx.obj
 0001:000083c1       _VEC3fromFix               100093c1 f   cmsmtrx.obj
 0001:000083e8       _VEC3swap                  100093e8 f   cmsmtrx.obj
 0001:00008411       _VEC3divK                  10009411 f   cmsmtrx.obj
 0001:00008434       _VEC3perK                  10009434 f   cmsmtrx.obj
 0001:00008458       _VEC3minus                 10009458 f   cmsmtrx.obj
 0001:000084a2       _VEC3equal                 100094a2 f   cmsmtrx.obj
 0001:000084f6       _VEC3saturate              100094f6 f   cmsmtrx.obj
 0001:0000852c       _MAT3identity              1000952c f   cmsmtrx.obj
 0001:0000855d       _MAT3per                   1000955d f   cmsmtrx.obj
 0001:00008644       _MAT3inverse               10009644 f   cmsmtrx.obj
 0001:00008803       _MAT3eval                  10009803 f   cmsmtrx.obj
 0001:00008856       _MAT3evalW                 10009856 f   cmsmtrx.obj
 0001:0000890c       _MAT3toFix                 1000990c f   cmsmtrx.obj
 0001:0000893d       _MAT3fromFix               1000993d f   cmsmtrx.obj
 0001:0000896c       _MAT3isIdentity            1000996c f   cmsmtrx.obj
 0001:000089c6       _MAT3solve                 100099c6 f   cmsmtrx.obj
 0001:00008aaa       _cmsAllocNamedColorList    10009aaa f   cmsnamed.obj
 0001:00008b01       _cmsFreeNamedColorList     10009b01 f   cmsnamed.obj
 0001:00008b20       _cmsAppendNamedColor       10009b20 f   cmsnamed.obj
 0001:0000a3c5       __cmsIdentifyInputFormat   1000b3c5 f   cmspack.obj
 0001:0000a767       __cmsIdentifyOutputFormat  1000b767 f   cmspack.obj
 0001:0000abe0       _cmsSetUserFormatters      1000bbe0 f   cmspack.obj
 0001:0000ac0d       _cmsChangeBuffersFormat    1000bc0d f   cmspack.obj
 0001:0000ad5a       _cmsXYZ2LabEncoded         1000bd5a f   cmspcs.obj
 0001:0000ae72       _cmsLab2XYZ                1000be72 f   cmspcs.obj
 0001:0000af11       _cmsLab2XYZEncoded         1000bf11 f   cmspcs.obj
 0001:0000b051       _cmsLabEncoded2Float       1000c051 f   cmspcs.obj
 0001:0000b09f       _cmsLabEncoded2Float4      1000c09f f   cmspcs.obj
 0001:0000b147       _cmsFloat2LabEncoded       1000c147 f   cmspcs.obj
 0001:0000b1d2       _cmsFloat2LabEncoded4      1000c1d2 f   cmspcs.obj
 0001:0000b2e2       _cmsFloat2XYZEncoded       1000c2e2 f   cmspcs.obj
 0001:0000b3be       _cmsXYZEncoded2Float       1000c3be f   cmspcs.obj
 0001:0000b402       __cmsQuantizeVal           1000c402 f   cmssamp.obj
 0001:0000b433       _cmsIsLinear               1000c433 f   cmssamp.obj
 0001:0000b47f       _cmsSample3DGrid           1000c47f f   cmssamp.obj
 0001:0000b64c       __cmsReasonableGridpointsByColorspace 1000c64c f   cmssamp.obj
 0001:0000b6d3       __cmsPrecalculateDeviceLink 1000c6d3 f   cmssamp.obj
 0001:0000ba7d       __cmsPrecalculateBlackPreservingDeviceLink 1000ca7d f   cmssamp.obj
 0001:0000be84       __cmsFixWhiteMisalignment  1000ce84 f   cmssamp.obj
 0001:0000bf04       _cmsCreateRGBProfile       1000cf04 f   cmsvirt.obj
 0001:0000c0b9       _cmsCreateLabProfile       1000d0b9 f   cmsvirt.obj
 0001:0000c16a       _cmsCreateXYZProfile       1000d16a f   cmsvirt.obj
 0001:0000c21f       _cmsXYZ2xyY                1000d21f f   cmswtpnt.obj
 0001:0000c248       _cmsxyY2XYZ                1000d248 f   cmswtpnt.obj
 0001:0000c271       _cmsBuildRGB2XYZtransferMatrix 1000d271 f   cmswtpnt.obj
 0001:0000c537       _cmsAdaptationMatrix       1000d537 f   cmswtpnt.obj
 0001:0000c5b1       _cmsAdaptMatrixToD50       1000d5b1 f   cmswtpnt.obj
 0001:0000c608       _cmsAdaptToIlluminant      1000d608 f   cmswtpnt.obj
 0001:0000c92f       _cmsDetectBlackPoint       1000d92f f   cmswtpnt.obj
 0001:0000d447       _cmsBuildInputMatrixShaper 1000e447 f   cmsxform.obj
 0001:0000d4da       _cmsBuildOutputMatrixShaper 1000e4da f   cmsxform.obj
 0001:0000ddb0       _cmsDeleteTransform        1000edb0 f   cmsxform.obj
 0001:0000de69       _cmsDoTransform            1000ee69 f   cmsxform.obj
 0001:0000de8b       __cmsIsMatrixShaper        1000ee8b f   cmsxform.obj
 0001:0000df23       _cmsIsIntentSupported      1000ef23 f   cmsxform.obj
 0001:0000e102       _cmsCreateProofingTransform 1000f102 f   cmsxform.obj
 0001:0000e4f4       _cmsCreateTransform        1000f4f4 f   cmsxform.obj
 0001:0000e517       _cmsCreateMultiprofileTransform 1000f517 f   cmsxform.obj
 0001:0000e967       _errorHandler              1000f967 f   LCMS.obj
 0001:0000e9a9       _JNI_OnLoad@8              1000f9a9 f   LCMS.obj
 0001:0000e9c5       _LCMS_freeTransform        1000f9c5 f   LCMS.obj
 0001:0000e9d0       _Java_sun_java2d_cmm_lcms_LCMS_createNativeTransform@20 1000f9d0 f   LCMS.obj
 0001:0000eb07       _Java_sun_java2d_cmm_lcms_LCMS_loadProfile@12 1000fb07 f   LCMS.obj
 0001:0000eb63       _Java_sun_java2d_cmm_lcms_LCMS_freeProfile@16 1000fb63 f   LCMS.obj
 0001:0000eba0       _Java_sun_java2d_cmm_lcms_LCMS_getProfileSize@16 1000fba0 f   LCMS.obj
 0001:0000ebe4       _Java_sun_java2d_cmm_lcms_LCMS_getProfileData@20 1000fbe4 f   LCMS.obj
 0001:0000ec68       _Java_sun_java2d_cmm_lcms_LCMS_getTagSize@20 1000fc68 f   LCMS.obj
 0001:0000ecb4       _Java_sun_java2d_cmm_lcms_LCMS_getTagData@24 1000fcb4 f   LCMS.obj
 0001:0000ed8a       _getILData                 1000fd8a f   LCMS.obj
 0001:0000ee0f       _releaseILData             1000fe0f f   LCMS.obj
 0001:0000ee78       _Java_sun_java2d_cmm_lcms_LCMS_colorConvert@20 1000fe78 f   LCMS.obj
 0001:0000f063       _Java_sun_java2d_cmm_lcms_LCMS_getProfileID@12 10010063 f   LCMS.obj
 0001:0000f07d       _Java_sun_java2d_cmm_lcms_LCMS_initLCMS@20 1001007d f   LCMS.obj
 0001:0000f1ad       __cmsModifyTagData         100101ad f   LCMS.obj
 0001:0000f5b2       _Java_sun_java2d_cmm_lcms_LCMS_setTagData@24 100105b2 f   LCMS.obj
 0001:0000f618       _JNU_ThrowByName@12        10010618 f   java:java.dll
 0001:0000f61e       _JNU_ThrowIllegalArgumentException@8 1001061e f   java:java.dll
 0001:0000f624       _Disposer_AddRecord@20     10010624 f   awt:awt.dll
 0001:0000f62a       _J2dTraceImpl              1001062a f   awt:awt.dll
 0001:0000f630       _pow                       10010630 f   MSVCRT:MSVCR71.dll
 0001:0000f636       _fabs                      10010636 f   MSVCRT:MSVCR71.dll
 0001:0000f63c       _memset                    1001063c f   MSVCRT:MSVCR71.dll
 0001:0000f642       _sqrt                      10010642 f   MSVCRT:MSVCR71.dll
 0001:0000f648       _strlen                    10010648 f   MSVCRT:MSVCR71.dll
 0001:0000f650       __ftol2                    10010650 f   MSVCRT:ftol2.obj
 0001:0000f6c6       _memcpy                    100106c6 f   MSVCRT:MSVCR71.dll
 0001:0000f6d0       __chkstk                   100106d0 f   MSVCRT:chkstk.obj
 0001:0000f6d0       __alloca_probe             100106d0     MSVCRT:chkstk.obj
 0001:0000f70e       _strcat                    1001070e f   MSVCRT:MSVCR71.dll
 0001:0000f714       _abs                       10010714 f   MSVCRT:MSVCR71.dll
 0001:0000f71a       _memcmp                    1001071a f   MSVCRT:MSVCR71.dll
 0001:0000f720       __CRT_INIT@12              10010720 f   MSVCRT:crtdll.obj
 0001:0000f7de       __DllMainCRTStartup@12     100107de f   MSVCRT:crtdll.obj
 0001:0000f8c2       __initterm                 100108c2 f   MSVCRT:MSVCR71.dll
 0001:0000f8c8       __onexit                   100108c8 f   MSVCRT:atonexit.obj
 0001:0000f8ee       _atexit                    100108ee f   MSVCRT:atonexit.obj
 0001:0000f900       __RTC_Initialize           10010900 f   MSVCRT:initsect.obj
 0001:0000f944       __RTC_Terminate            10010944 f   MSVCRT:initsect.obj
 0001:0000f988       ___CppXcptFilter           10010988 f   MSVCRT:MSVCR71.dll
 0001:0000f98e       _DllMain@12                1001098e f   MSVCRT:dllmain.obj
 0001:0000f9b0       __SEH_prolog               100109b0 f   MSVCRT:sehprolg.obj
 0001:0000f9eb       __SEH_epilog               100109eb f   MSVCRT:sehprolg.obj
 0001:0000f9fc       __except_handler3          100109fc f   MSVCRT:MSVCR71.dll
 0001:0000fa02       ___dllonexit               10010a02 f   MSVCRT:MSVCR71.dll
 0002:00000000       __imp__DisableThreadLibraryCalls@4 10011000     kernel32:KERNEL32.dll
 0002:00000004       __imp__FatalAppExitA@8     10011004     kernel32:KERNEL32.dll
 0002:00000008       \177KERNEL32_NULL_THUNK_DATA 10011008     kernel32:KERNEL32.dll
 0002:0000000c       __imp___onexit             1001100c     MSVCRT:MSVCR71.dll
 0002:00000010       __imp____dllonexit         10011010     MSVCRT:MSVCR71.dll
 0002:00000014       __imp___except_handler3    10011014     MSVCRT:MSVCR71.dll
 0002:00000018       __imp____CppXcptFilter     10011018     MSVCRT:MSVCR71.dll
 0002:0000001c       __imp__malloc              1001101c     MSVCRT:MSVCR71.dll
 0002:00000020       __imp__free                10011020     MSVCRT:MSVCR71.dll
 0002:00000024       __imp__pow                 10011024     MSVCRT:MSVCR71.dll
 0002:00000028       __imp__fabs                10011028     MSVCRT:MSVCR71.dll
 0002:0000002c       __imp__memset              1001102c     MSVCRT:MSVCR71.dll
 0002:00000030       __imp__sqrt                10011030     MSVCRT:MSVCR71.dll
 0002:00000034       __imp__strncpy             10011034     MSVCRT:MSVCR71.dll
 0002:00000038       __imp___snprintf           10011038     MSVCRT:MSVCR71.dll
 0002:0000003c       __imp___vsnprintf          1001103c     MSVCRT:MSVCR71.dll
 0002:00000040       __imp__fclose              10011040     MSVCRT:MSVCR71.dll
 0002:00000044       __imp___stricmp            10011044     MSVCRT:MSVCR71.dll
 0002:00000048       __imp__strlen              10011048     MSVCRT:MSVCR71.dll
 0002:0000004c       __imp__sprintf             1001104c     MSVCRT:MSVCR71.dll
 0002:00000050       __imp__memcpy              10011050     MSVCRT:MSVCR71.dll
 0002:00000054       __imp__fwrite              10011054     MSVCRT:MSVCR71.dll
 0002:00000058       __imp__fopen               10011058     MSVCRT:MSVCR71.dll
 0002:0000005c       __imp__strcat              1001105c     MSVCRT:MSVCR71.dll
 0002:00000060       __imp__floor               10011060     MSVCRT:MSVCR71.dll
 0002:00000064       __imp__abs                 10011064     MSVCRT:MSVCR71.dll
 0002:00000068       __imp__ceil                10011068     MSVCRT:MSVCR71.dll
 0002:0000006c       __imp__realloc             1001106c     MSVCRT:MSVCR71.dll
 0002:00000070       __imp___swab               10011070     MSVCRT:MSVCR71.dll
 0002:00000074       __imp__gmtime              10011074     MSVCRT:MSVCR71.dll
 0002:00000078       __imp__time                10011078     MSVCRT:MSVCR71.dll
 0002:0000007c       __imp___unlink             1001107c     MSVCRT:MSVCR71.dll
 0002:00000080       __imp__ldexp               10011080     MSVCRT:MSVCR71.dll
 0002:00000084       __imp__frexp               10011084     MSVCRT:MSVCR71.dll
 0002:00000088       __imp__memcmp              10011088     MSVCRT:MSVCR71.dll
 0002:0000008c       __imp___initterm           1001108c     MSVCRT:MSVCR71.dll
 0002:00000090       __imp___adjust_fdiv        10011090     MSVCRT:MSVCR71.dll
 0002:00000094       \177MSVCR71_NULL_THUNK_DATA 10011094     MSVCRT:MSVCR71.dll
 0002:00000098       __imp__MessageBoxA@16      10011098     user32:USER32.dll
 0002:0000009c       \177USER32_NULL_THUNK_DATA 1001109c     user32:USER32.dll
 0002:000000a0       __imp__Disposer_AddRecord@20 100110a0     awt:awt.dll
 0002:000000a4       __imp__J2dTraceImpl        100110a4     awt:awt.dll
 0002:000000a8       \177awt_NULL_THUNK_DATA    100110a8     awt:awt.dll
 0002:000000ac       __imp__JNU_ThrowIllegalArgumentException@8 100110ac     java:java.dll
 0002:000000b0       __imp__JNU_ThrowByName@12  100110b0     java:java.dll
 0002:000000b4       \177java_NULL_THUNK_DATA   100110b4     java:java.dll
 0002:000000e0       __real@3fe0000000000000    100110e0     cmscam02.obj
 0002:000000e8       __real@3fb999999999999a    100110e8     cmscam02.obj
 0002:000000f0       __real@3fd5555555555555    100110f0     cmscam02.obj
 0002:000000f8       __real@4000000000000000    100110f8     cmscam02.obj
 0002:00000100       __real@4014000000000000    10011100     cmscam02.obj
 0002:00000108       __real@3ff0000000000000    10011108     cmscam02.obj
 0002:00000110       __real@3f847ae147ae147b    10011110     cmscam02.obj
 0002:00000118       __real@0000000000000000    10011118     cmscam02.obj
 0002:00000120       __real@4069000000000000    10011120     cmscam02.obj
 0002:00000128       __real@4059000000000000    10011128     cmscam02.obj
 0002:00000130       __real@3fa3eab367a0f909    10011130     cmscam97.obj
 0002:00000138       __real@bfb189374bc6a7f0    10011138     cmscam97.obj
 0002:00000140       __real@3ff0793dd97f62b7    10011140     cmscam97.obj
 0002:00000148       __real@bfe801a36e2eb1c4    10011148     cmscam97.obj
 0002:00000150       __real@3ffb6a7ef9db22d1    10011150     cmscam97.obj
 0002:00000158       __real@3fa2ca57a786c227    10011158     cmscam97.obj
 0002:00000160       __real@3feca4a8c154c986    10011160     cmscam97.obj
 0002:00000168       __real@3fd10cb295e9e1b1    10011168     cmscam97.obj
 0002:00000170       __real@bfc4a8c154c985f0    10011170     cmscam97.obj
 0002:00000178       ??_C@_0M@CCEBNHDC@CHI_SQD_PAR?$AA@ 10011178     cmscgats.obj
 0002:00000184       ??_C@_08LCDEBKKI@STDEV_DE?$AA@ 10011184     cmscgats.obj
 0002:00000190       ??_C@_07NJPNJCCA@STDEV_B?$AA@ 10011190     cmscgats.obj
 0002:00000198       ??_C@_07PCNAMBOD@STDEV_A?$AA@ 10011198     cmscgats.obj
 0002:000001a0       ??_C@_07EHHOLPKO@STDEV_L?$AA@ 100111a0     cmscgats.obj
 0002:000001a8       ??_C@_07FLOGAKHJ@STDEV_Z?$AA@ 100111a8     cmscgats.obj
 0002:000001b0       ??_C@_07HAMLFJLK@STDEV_Y?$AA@ 100111b0     cmscgats.obj
 0002:000001b8       ??_C@_07GJNAGIPL@STDEV_X?$AA@ 100111b8     cmscgats.obj
 0002:000001c0       ??_C@_07HEECBDDN@MEAN_DE?$AA@ 100111c0     cmscgats.obj
 0002:000001c8       ??_C@_0M@HPKLADL@LAB_DE_2000?$AA@ 100111c8     cmscgats.obj
 0002:000001d4       ??_C@_0L@DKBFAEGH@LAB_DE_CMC?$AA@ 100111d4     cmscgats.obj
 0002:000001e0       ??_C@_09OIBLJGHC@LAB_DE_94?$AA@ 100111e0     cmscgats.obj
 0002:000001ec       ??_C@_06GOPMGMME@LAB_DE?$AA@ 100111ec     cmscgats.obj
 0002:000001f4       ??_C@_05DNGJNJIE@LAB_H?$AA@ 100111f4     cmscgats.obj
 0002:000001fc       ??_C@_05NOJNAAEP@LAB_C?$AA@ 100111fc     cmscgats.obj
 0002:00000204       ??_C@_05MHIGDBAO@LAB_B?$AA@ 10011204     cmscgats.obj
 0002:0000020c       ??_C@_05OMKLGCMN@LAB_A?$AA@ 1001120c     cmscgats.obj
 0002:00000214       ??_C@_05FJAFBMIA@LAB_L?$AA@ 10011214     cmscgats.obj
 0002:0000021c       ??_C@_08OKLOCDPI@XYY_CAPY?$AA@ 1001121c     cmscgats.obj
 0002:00000228       ??_C@_0L@DOILIGPP@XYY_XXYY_Y?$AA@ 10011228     cmscgats.obj
 0002:00000234       ??_C@_05BIOHEKOJ@XYZ_Z?$AA@ 10011234     cmscgats.obj
 0002:0000023c       ??_C@_05DDMKBJCK@XYZ_Y?$AA@ 1001123c     cmscgats.obj
 0002:00000244       ??_C@_05CKNBCIGL@XYZ_X?$AA@ 10011244     cmscgats.obj
 0002:0000024c       ??_C@_0N@LEJCFEG@SPECTRAL_DEC?$AA@ 1001124c     cmscgats.obj
 0002:0000025c       ??_C@_0N@NFDMBNKK@SPECTRAL_PCT?$AA@ 1001125c     cmscgats.obj
 0002:0000026c       ??_C@_0M@LIGBHIDL@SPECTRAL_NM?$AA@ 1001126c     cmscgats.obj
 0002:00000278       ??_C@_05HBBKKHEF@RGB_B?$AA@ 10011278     cmscgats.obj
 0002:00000280       ??_C@_05MGNFDAA@RGB_G?$AA@ 10011280     cmscgats.obj
 0002:00000288       ??_C@_05DLNILFBE@RGB_R?$AA@ 10011288     cmscgats.obj
 0002:00000290       ??_C@_0P@OLJLEEFM@D_MAJOR_FILTER?$AA@ 10011290     cmscgats.obj
 0002:000002a0       ??_C@_05GAAMKGJK@D_VIS?$AA@ 100112a0     cmscgats.obj
 0002:000002a8       ??_C@_06DLIHHAHO@D_BLUE?$AA@ 100112a8     cmscgats.obj
 0002:000002b0       ??_C@_07GHIFGAP@D_GREEN?$AA@ 100112b0     cmscgats.obj
 0002:000002b8       ??_C@_05ODPHEMDP@D_RED?$AA@ 100112b8     cmscgats.obj
 0002:000002c0       ??_C@_06KJMNNLBC@CMYK_K?$AA@ 100112c0     cmscgats.obj
 0002:000002c8       ??_C@_06NBDJKLMB@CMYK_Y?$AA@ 100112c8     cmscgats.obj
 0002:000002d0       ??_C@_06PPJHHMJE@CMYK_M?$AA@ 100112d0     cmscgats.obj
 0002:000002d8       ??_C@_06GBBEFBBK@CMYK_C?$AA@ 100112d8     cmscgats.obj
 0002:000002e0       ??_C@_06IGECGLFO@STRING?$AA@ 100112e0     cmscgats.obj
 0002:000002e8       ??_C@_09IGELLNJJ@SAMPLE_ID?$AA@ 100112e8     cmscgats.obj
 0002:000002f4       ??_C@_0L@HJPNOMFH@TABLE_NAME?$AA@ 100112f4     cmscgats.obj
 0002:00000300       ??_C@_0BB@IJIAOGIB@TABLE_DESCRIPTOR?$AA@ 10011300     cmscgats.obj
 0002:00000314       ??_C@_08LGFJDIAP@COLORANT?$AA@ 10011314     cmscgats.obj
 0002:00000320       ??_C@_0M@HKJIKBKL@TARGET_TYPE?$AA@ 10011320     cmscgats.obj
 0002:0000032c       ??_C@_0BI@LGGFFBDK@COMPUTATIONAL_PARAMETER?$AA@ 1001132c     cmscgats.obj
 0002:00000344       ??_C@_0BD@PMHFGOKD@WEIGHTING_FUNCTION?$AA@ 10011344     cmscgats.obj
 0002:00000358       ??_C@_0N@BLIEIPH@POLARIZATION?$AA@ 10011358     cmscgats.obj
 0002:00000368       ??_C@_06EKKPGGCG@FILTER?$AA@ 10011368     cmscgats.obj
 0002:00000370       ??_C@_0BF@BFDKHDLE@MEASUREMENT_GEOMETRY?$AA@ 10011370     cmscgats.obj
 0002:00000388       ??_C@_09JMFPMOIF@CHISQ_DOF?$AA@ 10011388     cmscgats.obj
 0002:00000394       ??_C@_0P@KIIFMCBO@SAMPLE_BACKING?$AA@ 10011394     cmscgats.obj
 0002:000003a4       ??_C@_0BB@CCJPNIDB@PRINT_CONDITIONS?$AA@ 100113a4     cmscgats.obj
 0002:000003b8       ??_C@_0BD@EJAFHPHI@MEASUREMENT_SOURCE?$AA@ 100113b8     cmscgats.obj
 0002:000003cc       ??_C@_0BA@GCECPBPC@INSTRUMENTATION?$AA@ 100113cc     cmscgats.obj
 0002:000003dc       ??_C@_08NCEIPHOL@MATERIAL?$AA@ 100113dc     cmscgats.obj
 0002:000003e8       ??_C@_06KGGACEJG@SERIAL?$AA@ 100113e8     cmscgats.obj
 0002:000003f0       ??_C@_09CMIELPMF@PROD_DATE?$AA@ 100113f0     cmscgats.obj
 0002:000003fc       ??_C@_0M@NCKCGAOL@MANUFACTURE?$AA@ 100113fc     cmscgats.obj
 0002:00000408       ??_C@_0N@LPIHKGEG@MANUFACTURER?$AA@ 10011408     cmscgats.obj
 0002:00000418       ??_C@_0BB@FHCOAJ@DIFFUSE_GEOMETRY?$AA@ 10011418     cmscgats.obj
 0002:0000042c       ??_C@_0L@HFJNFBAI@DESCRIPTOR?$AA@ 1001142c     cmscgats.obj
 0002:00000438       ??_C@_07BFKIKKPP@CREATED?$AA@ 10011438     cmscgats.obj
 0002:00000440       ??_C@_0BA@LGMGNJKE@FILE_DESCRIPTOR?$AA@ 10011440     cmscgats.obj
 0002:00000450       ??_C@_0L@LDGMMHG@ORIGINATOR?$AA@ 10011450     cmscgats.obj
 0002:0000045c       ??_C@_0P@DOAEDAOK@NUMBER_OF_SETS?$AA@ 1001145c     cmscgats.obj
 0002:0000046c       ??_C@_0BB@HDJDLEKM@NUMBER_OF_FIELDS?$AA@ 1001146c     cmscgats.obj
 0002:000004c0       ??_C@_07GBPBNGKD@KEYWORD?$AA@ 100114c0     cmscgats.obj
 0002:000004c8       ??_C@_0BA@JKEAGHEK@END_DATA_FORMAT?$AA@ 100114c8     cmscgats.obj
 0002:000004d8       ??_C@_08PAHEKPHH@END_DATA?$AA@ 100114d8     cmscgats.obj
 0002:000004e4       ??_C@_0BH@BKLCBPCO@DATA_FORMAT_IDENTIFIER?$AA@ 100114e4     cmscgats.obj
 0002:000004fc       ??_C@_0BC@MJMHIBCL@BEGIN_DATA_FORMAT?$AA@ 100114fc     cmscgats.obj
 0002:00000510       ??_C@_0L@LAOBICO@BEGIN_DATA?$AA@ 10011510     cmscgats.obj
 0002:0000051c       ??_C@_08GDKCMJME@?4INCLUDE?$AA@ 1001151c     cmscgats.obj
 0002:00000528       ??_C@_08PGIMEDFK@$INCLUDE?$AA@ 10011528     cmscgats.obj
 0002:00000531       ??_C@_00CNPNBAHC@?$AA@     10011531     cmscgats.obj
 0002:00000538       __real@3ee4f8b588e368f1    10011538     cmscnvrt.obj
 0002:00000540       ??_C@_0BH@ILOLDAME@?$CIinternal?$CJ?5Phase?5error?$AA@ 10011540     cmscnvrt.obj
 0002:00000558       ??_C@_0CA@LHEOCBHI@lcms?5is?5terminating?5application?$AA@ 10011558     cmserr.obj
 0002:00000578       ??_C@_0L@FIONFKOF@Little?5cms?$AA@ 10011578     cmserr.obj
 0002:00000584       ??_C@_0M@EBCCNHKP@Error?5?$CD?$CFx?$DL?5?$AA@ 10011584     cmserr.obj
 0002:00000590       ??_C@_0DG@FHGMHNKL@Couldn?8t?5create?5gammatable?5of?5mo@ 10011590     cmsgamma.obj
 0002:000005c8       ??_C@_0CF@IJMOMLOJ@Unsupported?5parametric?5curve?5typ@ 100115c8     cmsgamma.obj
 0002:000005f0       __real@40efffe000000000    100115f0     cmsgamma.obj
 0002:000005f8       __real@3ef0001000100010    100115f8     cmsgamma.obj
 0002:00000600       __real@40f0000000000000    10011600     cmsgamma.obj
 0002:00000608       ??_C@_0DK@CHODIJKE@cmsConvertGammaToSampledCurve?3?5t@ 10011608     cmsgamma.obj
 0002:00000648       __real@3f50624dd2f1a9fc    10011648     cmsgamma.obj
 0002:00000650       __real@c069000000000000    10011650     cmsgmt.obj
 0002:00000658       __real@3f81a7b9611a7b96    10011658     cmsgmt.obj
 0002:00000660       __real@4030000000000000    10011660     cmsgmt.obj
 0002:00000668       __real@4049000000000000    10011668     cmsgmt.obj
 0002:00000670       __real@4238000000008000    10011670     cmsgmt.obj
 0002:00000678       __real@3f947ae147ae147b    10011678     cmsgmt.obj
 0002:00000680       __real@41f0000000000000    10011680     cmsgmt.obj
 0002:00000688       ??_C@_0CG@OLBEKMDM@Unsupported?5restoration?5?$CI?$CFd?5chan@ 10011688     cmsintrp.obj
 0002:000006b0       ??_C@_0DD@GFOHOCLG@Read?5from?5memory?5error?4?5Integer?5@ 100116b0     cmsio0.obj
 0002:000006e8       ??_C@_0EC@HENBOIOF@Read?5from?5memory?5error?4?5Got?5?$CFd?5b@ 100116e8     cmsio0.obj
 0002:0000072c       ??_C@_0DM@GJAJNLNN@Read?5from?5memory?5error?4?5Integer?5@ 1001172c     cmsio0.obj
 0002:00000768       ??_C@_0CH@OCMNFIJ@Pointer?5error?$DL?5probably?5corrupte@ 10011768     cmsio0.obj
 0002:00000790       ??_C@_0BE@HDBKKJFO@Tag?5?8?$CFlx?8?5not?5found?$AA@ 10011790     cmsio0.obj
 0002:000007a4       ??_C@_0BD@JMMMDFNL@Too?5many?5tags?5?$CI?$CFd?$CJ?$AA@ 100117a4     cmsio0.obj
 0002:000007b8       ??_C@_0CI@FBACEILJ@Couldn?8t?5allocate?5?$CFld?5bytes?5for?5@ 100117b8     cmsio0.obj
 0002:000007e0       ??_C@_0BM@JICOGBFB@Couldn?8t?5write?5to?5file?5?8?$CFs?8?$AA@ 100117e0     cmsio0.obj
 0002:000007fc       ??_C@_02GMLFBBN@wb?$AA@    100117fc     cmsio0.obj
 0002:00000800       __real@3f70000000000000    10011800     cmsio1.obj
 0002:00000808       __real@3ef0000000000000    10011808     cmsio1.obj
 0002:00000810       ??_C@_0BI@FIBKNNFP@Corrupted?5profile?3?5?8?$CFs?8?$AA@ 10011810     cmsio1.obj
 0002:00000828       ??_C@_0BJ@MOJBCLPN@Corrupted?5memory?5profile?$AA@ 10011828     cmsio1.obj
 0002:00000848       __real@3ff0100000000000    10011848     cmsio1.obj
 0002:00000850       __real@3f1a36e2eb1c432d    10011850     cmsio1.obj
 0002:00000858       ??_C@_0CK@OBIOHCME@Unknown?5parametric?5curve?5type?5?8?$CF@ 10011858     cmsio1.obj
 0002:00000884       ??_C@_0BP@MNFACBDG@Bad?5tag?5signature?5?8?$CFlx?8?5found?4?$AA@ 10011884     cmsio1.obj
 0002:000008a4       ??_C@_0BK@OIMKOOLO@Unknow?5precission?5of?5?8?$CFd?8?$AA@ 100118a4     cmsio1.obj
 0002:000008c0       ??_C@_0DK@PEHNLGBD@CLUT?5with?5different?5granulatity?5@ 100118c0     cmsio1.obj
 0002:000008fc       ??_C@_0BN@EGOGCGFK@Bad?5tag?5signature?5?$CFlx?5found?4?$AA@ 100118fc     cmsio1.obj
 0002:0000091c       ??_C@_0BF@GOPNGLCD@cmsAllocLUT?$CI?$CJ?5failed?$AA@ 1001191c     cmsio1.obj
 0002:00000934       ??_C@_0BO@MKKKBNFP@Bad?5array?5size?5of?5?$CFd?5entries?4?$AA@ 10011934     cmsio1.obj
 0002:00000954       ??_C@_0BN@IGFJKNGK@Too?5many?5device?5coordinates?4?$AA@ 10011954     cmsio1.obj
 0002:00000974       ??_C@_0DI@PDLNDJPB@prefix?1suffix?1device?5for?5named?5c@ 10011974     cmsio1.obj
 0002:000009ac       ??_C@_0DA@NCOOAJNN@Ancient?5named?5color?5profiles?5are@ 100119ac     cmsio1.obj
 0002:000009e0       __real@3f6fe01fe01fe020    100119e0     cmsio1.obj
 0002:000009e8       ??_C@_0CM@FOIOMMKC@LUT8?5needs?5256?5entries?5on?5postli@ 100119e8     cmsio1.obj
 0002:00000a14       ??_C@_0CL@PJACHFCE@LUT8?5needs?5256?5entries?5on?5prelin@ 10011a14     cmsio1.obj
 0002:00000a40       ??_C@_0CD@FDMBBDDP@cmsAddTag?3?5Tag?5?8?$CFx?8?5is?5unsupport@ 10011a40     cmsio1.obj
 0002:00000a68       __real@3feff7ced916872b    10011a68     cmslut.obj
 0002:00000a70       __real@408f400000000000    10011a70     cmslut.obj
 0002:00000a78       __real@3fd3333333333333    10011a78     cmslut.obj
 0002:00000a80       __real@4415af1d78b58c40    10011a80     cmslut.obj
 0002:00000a88       ??_C@_0CM@JNAOANJD@Out?5of?5memory?5reallocating?5named@ 10011a88     cmsnamed.obj
 0002:00000ab4       ??_C@_0CI@NCBFIGPJ@Out?5of?5memory?5creating?5named?5col@ 10011ab4     cmsnamed.obj
 0002:00000adc       ??_C@_0CG@OMLCOFED@Couldn?8t?5free?5a?5NULL?5named?5color@ 10011adc     cmsnamed.obj
 0002:00000b08       __real@40847acccccccccd    10011b08     cmspack.obj
 0002:00000b10       __real@3f59001900190019    10011b10     cmspack.obj
 0002:00000b18       ??_C@_0BF@NLMPEOMC@Unknown?5input?5format?$AA@ 10011b18     cmspack.obj
 0002:00000b30       ??_C@_0CJ@PDKPINOL@Named?5color?5needs?5TYPE_NAMED_COL@ 10011b30     cmspack.obj
 0002:00000b5c       ??_C@_0BG@FAGKCPBK@Unknown?5output?5format?$AA@ 10011b5c     cmspack.obj
 0002:00000b78       __real@4040fecbc9e2c375    10011b78     cmspcs.obj
 0002:00000b80       __real@406510d06a8112ce    10011b80     cmspcs.obj
 0002:00000b88       __real@4062ff15c0285815    10011b88     cmspcs.obj
 0002:00000b90       __real@402d9e20660edb21    10011b90     cmspcs.obj
 0002:00000b98       __real@3fc4f15f83f55d2d    10011b98     cmspcs.obj
 0002:00000ba0       __real@402add70d2827500    10011ba0     cmspcs.obj
 0002:00000ba8       __real@405dca97439cae14    10011ba8     cmspcs.obj
 0002:00000bb0       __real@406808f46c6116e0    10011bb0     cmspcs.obj
 0002:00000bb8       __real@4046a09e6653ba70    10011bb8     cmspcs.obj
 0002:00000bc0       __real@3fc1a7b9611a7b96    10011bc0     cmspcs.obj
 0002:00000bc8       __real@401f25ed097b425f    10011bc8     cmspcs.obj
 0002:00000bd0       __real@3f822354d28f7cd6    10011bd0     cmspcs.obj
 0002:00000bd8       __real@3fc07004ded20922    10011bd8     cmspcs.obj
 0002:00000be0       __real@3fca7b9611a7b961    10011be0     cmspcs.obj
 0002:00000be8       __real@407f400000000000    10011be8     cmspcs.obj
 0002:00000bf0       __real@405d000000000000    10011bf0     cmspcs.obj
 0002:00000bf8       __real@4084666666666666    10011bf8     cmspcs.obj
 0002:00000c00       __real@4070000000000000    10011c00     cmspcs.obj
 0002:00000c08       __real@4060000000000000    10011c08     cmspcs.obj
 0002:00000c10       __real@3ff365734aa30d90    10011c10     cmspcs.obj
 0002:00000c18       __real@3ff09814d0cb0eec    10011c18     cmspcs.obj
 0002:00000c20       __real@3f60624dd2f1a9fc    10011c20     cmspcs.obj
 0002:00000c28       __real@3f747ae147ae147b    10011c28     cmspcs.obj
 0002:00000c30       __real@40e0000000000000    10011c30     cmspcs.obj
 0002:00000c38       __real@3fea6594af4f0d84    10011c38     cmspcs.obj
 0002:00000c40       __real@3feedab9f559b3d0    10011c40     cmspcs.obj
 0002:00000c48       __real@3ef0101010101010    10011c48     cmspcs.obj
 0002:00000c50       __real@3f5919191919191a    10011c50     cmspcs.obj
 0002:00000c58       __real@4070100000000000    10011c58     cmspcs.obj
 0002:00000c60       __real@405fffc01a36e2eb    10011c60     cmspcs.obj
 0002:00000c68       __real@c060000000000000    10011c68     cmspcs.obj
 0002:00000c70       __real@405fc00000000000    10011c70     cmspcs.obj
 0002:00000c78       __real@3fffffd60e94ee39    10011c78     cmspcs.obj
 0002:00000c94       ??_C@_0DF@HOPCOCIH@?$CIinternal?$CJ?5?$CFd?5Channels?5are?5not?5s@ 10011c94     cmssamp.obj
 0002:00000ccc       ??_C@_0N@CEEDKOLH@rgb?5built?9in?$AA@ 10011ccc     cmsvirt.obj
 0002:00000cdc       ??_C@_0BJ@JAPCEHDK@lcms?5RGB?5virtual?5profile?$AA@ 10011cdc     cmsvirt.obj
 0002:00000cf8       ??_C@_0BA@LCLGKBBF@?$CIlcms?5internal?$CJ?$AA@ 10011cf8     cmsvirt.obj
 0002:00000d08       ??_C@_0N@DGOBOKMI@Lab?5built?9in?$AA@ 10011d08     cmsvirt.obj
 0002:00000d18       ??_C@_0BC@NCKKMGMM@lcms?5Lab?5identity?$AA@ 10011d18     cmsvirt.obj
 0002:00000d2c       ??_C@_0N@MCNDMMCH@XYZ?5built?9in?$AA@ 10011d2c     cmsvirt.obj
 0002:00000d3c       ??_C@_0BC@CGJIOACD@lcms?5XYZ?5identity?$AA@ 10011d3c     cmsvirt.obj
 0002:00000d50       __real@3f6782d38476f2a6    10011d50     cmswtpnt.obj
 0002:00000d58       __real@3f6c739e5d4db8f0    10011d58     cmswtpnt.obj
 0002:00000d60       __real@3f6b866e43aa79bc    10011d60     cmswtpnt.obj
 0002:00000d68       ??_C@_0BG@HHNOOACC@Color?5?$CFd?5out?5of?5range?$AA@ 10011d68     cmsxform.obj
 0002:00000d80       ??_C@_0M@HIIEIFNB@Invalid?5PCS?$AA@ 10011d80     cmsxform.obj
 0002:00000d8c       ??_C@_0CI@CGEMBFBJ@cmsCreateTransform?3?5_cmsMalloc?$CI?$CJ@ 10011d8c     cmsxform.obj
 0002:00000db4       ??_C@_0DN@PIBBGKMM@Sorry?0?5the?5proof?5profile?5has?5not@ 10011db4     cmsxform.obj
 0002:00000df4       ??_C@_0DJ@FBHLNDEB@Sorry?0?5the?5proof?5profile?5has?5not@ 10011df4     cmsxform.obj
 0002:00000e30       ??_C@_0CB@HNOJPKGH@profile?5is?5unsuitable?5for?5output@ 10011e30     cmsxform.obj
 0002:00000e54       ??_C@_0CA@OINHECNJ@profile?5is?5unsuitable?5for?5input?$AA@ 10011e54     cmsxform.obj
 0002:00000e74       ??_C@_0DF@GKGJPMCK@unable?5to?5smelt?5shaper?9matrix?0?5r@ 10011e74     cmsxform.obj
 0002:00000eac       ??_C@_0BK@HHCHMIIC@Unexpected?5direction?5?$CI?$CFd?$CJ?$AA@ 10011eac     cmsxform.obj
 0002:00000ec8       ??_C@_0EF@LLOJDIOL@Output?5profile?5should?5be?5NULL?0?5s@ 10011ec8     cmsxform.obj
 0002:00000f10       ??_C@_0DB@NMPMGPBN@Proofing?5not?5supported?5on?5device@ 10011f10     cmsxform.obj
 0002:00000f44       ??_C@_0CB@ODLJGCLK@Noncompliant?5device?9link?5profile@ 10011f44     cmsxform.obj
 0002:00000f68       ??_C@_0DH@EIJCJAKJ@Device?5link?5is?5operating?5on?5wron@ 10011f68     cmsxform.obj
 0002:00000fa0       ??_C@_0DG@CGBFHGPB@Device?5link?5is?5operating?5on?5wron@ 10011fa0     cmsxform.obj
 0002:00000fd8       ??_C@_0CE@EOMMNBPP@cmsCreateTransform?3?5intent?5misma@ 10011fd8     cmsxform.obj
 0002:00000ffc       ??_C@_0CP@DCLMPBBF@Cannot?5precalculate?5?$CFd?9?$DO?$CFd?5chann@ 10011ffc     cmsxform.obj
 0002:0000102c       ??_C@_0DB@BHBCENDD@Named?5color?5profiles?5are?5not?5sup@ 1001202c     cmsxform.obj
 0002:00001060       ??_C@_0DA@ICHJDPNA@Output?5profile?5is?5operating?5on?5w@ 10012060     cmsxform.obj
 0002:00001090       ??_C@_0BP@HGLGPKGF@Output?5profile?5cannot?5be?5NULL?$CB?$AA@ 10012090     cmsxform.obj
 0002:000010b0       ??_C@_0CP@LJPAACIE@Input?5profile?5is?5operating?5on?5wr@ 100120b0     cmsxform.obj
 0002:000010e0       ??_C@_0BO@PJPBKANF@Input?5profile?5cannot?5be?5NULL?$CB?$AA@ 100120e0     cmsxform.obj
 0002:00001100       ??_C@_0DE@ECPCLKLF@cmsCreateMultiprofileTransform?3?5@ 10012100     cmsxform.obj
 0002:00001134       ??_C@_0DL@FGGICCJL@cmsCreateMultiprofileTransform?3?5@ 10012134     cmsxform.obj
 0002:00001170       ??_C@_0EO@EGKILAGK@Could?5not?5mix?5named?5color?5profil@ 10012170     cmsxform.obj
 0002:000011c0       ??_C@_0EM@MCAJOPCN@What?5are?5you?5trying?5to?5do?5with?5m@ 100121c0     cmsxform.obj
 0002:0000120c       ??_C@_0BM@DKJNFALL@java?1awt?1color?1CMMException?$AA@ 1001220c     LCMS.obj
 0002:00001228       ??_C@_0O@CDGBALNI@LCMS?5error?5?$CFd?$AA@ 10012228     LCMS.obj
 0002:00001238       ??_C@_0BL@NGONHNHM@Cannot?5get?5color?5transform?$AA@ 10012238     LCMS.obj
 0002:00001254       ??_C@_0CO@CFOLACOL@LCMS_createNativeTransform?3?5sTra@ 10012254     LCMS.obj
 0002:00001284       ??_C@_0BL@NCIANLHP@getXForm?3?5iccArray?5?$DN?$DN?5NULL?$AA@ 10012284     LCMS.obj
 0002:000012a0       ??_C@_0BF@CIGEDMAF@Invalid?5profile?5data?$AA@ 100122a0     LCMS.obj
 0002:000012b8       ??_C@_0BF@IHFHPEAB@Cannot?5close?5profile?$AA@ 100122b8     LCMS.obj
 0002:000012d0       ??_C@_0CK@GHNIDFGO@LCMS_freeProfile?3?5cmsCloseProfil@ 100122d0     LCMS.obj
 0002:000012fc       ??_C@_0BK@OPEDDCAA@ICC?5profile?5tag?5not?5found?$AA@ 100122fc     LCMS.obj
 0002:00001318       ??_C@_0BH@PNOACLGC@Cannot?5get?5output?5data?$AA@ 10012318     LCMS.obj
 0002:00001330       ??_C@_0BG@BMANGOIB@Cannot?5get?5input?5data?$AA@ 10012330     LCMS.obj
 0002:00001348       ??_C@_0CF@MCBLFNBG@LCMS_colorConvert?3?5transform?5?$DN?$DN?5@ 10012348     LCMS.obj
 0002:00001370       ??_C@_0O@IIJELCFP@nextRowOffset?$AA@ 10012370     LCMS.obj
 0002:00001380       ??_C@_06KLHHMIGM@offset?$AA@ 10012380     LCMS.obj
 0002:00001388       ??_C@_06LNLHEAAG@height?$AA@ 10012388     LCMS.obj
 0002:00001390       ??_C@_05IGKADHGO@width?$AA@ 10012390     LCMS.obj
 0002:00001398       ??_C@_09LLHCBPIG@dataArray?$AA@ 10012398     LCMS.obj
 0002:000013a4       ??_C@_0BD@HMGGFBMH@Ljava?1lang?1Object?$DL?$AA@ 100123a4     LCMS.obj
 0002:000013b8       ??_C@_09FECOHCAH@pixelType?$AA@ 100123b8     LCMS.obj
 0002:000013c4       ??_C@_08EIGIMCLE@dataType?$AA@ 100123c4     LCMS.obj
 0002:000013d0       ??_C@_0M@BFEAFNHC@isIntPacked?$AA@ 100123d0     LCMS.obj
 0002:000013dc       ??_C@_01POHCFINO@Z?$AA@    100123dc     LCMS.obj
 0002:000013e0       ??_C@_02OLOABKKD@ID?$AA@   100123e0     LCMS.obj
 0002:000013e4       ??_C@_01LELAEKIP@J?$AA@    100123e4     LCMS.obj
 0002:000013e8       ??_C@_0L@MNEDCAEF@renderType?$AA@ 100123e8     LCMS.obj
 0002:000013f4       ??_C@_01JPJNBJEM@I?$AA@    100123f4     LCMS.obj
 0002:000013f8       ??_C@_0L@KIOPIILI@profileIDs?$AA@ 100123f8     LCMS.obj
 0002:00001404       ??_C@_02GKMBEADD@?$FLJ?$AA@ 10012404     LCMS.obj
 0002:00001408       ??_C@_0CI@LABOJMED@_cmsModifyTagData?3?5Icc?9?$DOGrow?$CI?$CJ?5?$DN@ 10012408     LCMS.obj
 0002:00001430       ??_C@_0CE@LHGPAMJL@_cmsModifyTagData?3?5afterBuf?5?$DN?$DN?5N@ 10012430     LCMS.obj
 0002:00001454       ??_C@_0CF@NNGHAKEL@_cmsModifyTagData?3?5beforeBuf?5?$DN?$DN?5@ 10012454     LCMS.obj
 0002:0000147c       ??_C@_0BP@NNAOPMJH@_cmsModifyTagData?3?5ptr?5?$DN?$DN?5NULL?$AA@ 1001247c     LCMS.obj
 0002:0000149c       ??_C@_0CH@NECPDGCP@_cmsModifyTagData?3?5Too?5many?5tags@ 1001249c     LCMS.obj
 0002:000014c4       ??_C@_0CL@GCBDOLJB@LCMS_setTagData?5on?5icSigHead?5not@ 100124c4     LCMS.obj
 0002:00001520       __load_config_used         10012520     MSVCRT:loadcfg.obj
 0002:000015d0       ___safe_se_handler_table   100125d0     <linker-defined>
 0002:000015d4       ___rtc_iaa                 100125d4     MSVCRT:initsect.obj
 0002:000015d8       ___rtc_izz                 100125d8     MSVCRT:initsect.obj
 0002:000015dc       ___rtc_taa                 100125dc     MSVCRT:initsect.obj
 0002:000015e0       ___rtc_tzz                 100125e0     MSVCRT:initsect.obj
 0002:000015e4       __IMPORT_DESCRIPTOR_java   100125e4     java:java.dll
 0002:000015f8       __IMPORT_DESCRIPTOR_USER32 100125f8     user32:USER32.dll
 0002:0000160c       __IMPORT_DESCRIPTOR_awt    1001260c     awt:awt.dll
 0002:00001620       __IMPORT_DESCRIPTOR_MSVCR71 10012620     MSVCRT:MSVCR71.dll
 0002:00001634       __IMPORT_DESCRIPTOR_KERNEL32 10012634     kernel32:KERNEL32.dll
 0002:00001648       __NULL_IMPORT_DESCRIPTOR   10012648     java:java.dll
 0003:00000000       ___xc_a                    10013000     MSVCRT:cinitexe.obj
 0003:00000004       ___xc_z                    10013004     MSVCRT:cinitexe.obj
 0003:00000008       ___xi_a                    10013008     MSVCRT:cinitexe.obj
 0003:0000000c       ___xi_z                    1001300c     MSVCRT:cinitexe.obj
 0003:00000600       ___security_cookie         10013600     MSVCRT:seccook.obj
 0003:000030fc       _javaVM                    100160fc     <common>
 0003:00003100       __adjust_fdiv              10016100     <common>
 0003:00003104       ___onexitend               10016104     <common>
 0003:00003108       ___onexitbegin             10016108     <common>
 0003:0000310c       __pRawDllMain              1001610c     <common>

 entry point at        0001:0000f7de

 Static symbols

 0001:00000049       _Rel2RelStepAbsCoefs       10001049 f   cmscnvrt.obj
 0001:000001b4       _ComputeBlackPointCompensationFactors 100011b4 f   cmscnvrt.obj
 0001:00000293       _IdentityParameters        10001293 f   cmscnvrt.obj
 0001:000002f5       _XYZ2XYZ                   100012f5 f   cmscnvrt.obj
 0001:0000036b       _XYZ2Lab                   1000136b f   cmscnvrt.obj
 0001:00000393       _Lab2XYZ                   10001393 f   cmscnvrt.obj
 0001:000003bb       _Lab2XYZ2Lab               100013bb f   cmscnvrt.obj
 0001:000003f1       _FromXYZRelLUT             100013f1 f   cmscnvrt.obj
 0001:000004ca       _FromLabRelLUT             100014ca f   cmscnvrt.obj
 0001:0000076d       _Crc32                     1000176d f   cmsgamma.obj
 0001:00000d0b       _ScaleVal                  10001d0b f   cmsgamma.obj
 0001:00001488       _CreateLabPrelinearization 10002488 f   cmsgmt.obj
 0001:000014e1       _GamutSampler              100024e1 f   cmsgmt.obj
 0001:00001660       _ComputeGamutWithInput     10002660 f   cmsgmt.obj
 0001:00001824       _SoftProofSampler          10002824 f   cmsgmt.obj
 0001:0000194a       _SlopeLimiting             1000294a f   cmsgmt.obj
 0001:000019be       _IsMonotonic               100029be f   cmsgmt.obj
 0001:00001c1e       _ComputeKToLstar           10002c1e f   cmsgmt.obj
 0001:00001d51       _Eval1Input                10002d51 f   cmsintrp.obj
 0001:000028e9       _Eval4Inputs               100038e9 f   cmsintrp.obj
 0001:000029a2       _Eval5Inputs               100039a2 f   cmsintrp.obj
 0001:00002a5b       _Eval6Inputs               10003a5b f   cmsintrp.obj
 0001:00002b14       _Eval7Inputs               10003b14 f   cmsintrp.obj
 0001:00002bcd       _Eval8Inputs               10003bcd f   cmsintrp.obj
 0001:00002d71       _MemoryOpen                10003d71 f   cmsio0.obj
 0001:00002dda       _MemoryRead                10003dda f   cmsio0.obj
 0001:00002e64       _MemorySeek                10003e64 f   cmsio0.obj
 0001:00002e8e       _MemoryTell                10003e8e f   cmsio0.obj
 0001:00002e98       _MemoryWrite               10003e98 f   cmsio0.obj
 0001:00002ed0       _MemoryGrow                10003ed0 f   cmsio0.obj
 0001:00002f06       _MemoryClose               10003f06 f   cmsio0.obj
 0001:00002f2d       _FileWrite                 10003f2d f   cmsio0.obj
 0001:00002f61       _FileClose                 10003f61 f   cmsio0.obj
 0001:0000324a       _DupBlock                  1000424a f   cmsio0.obj
 0001:0000344a       _AdjustEndianess32         1000444a f   cmsio1.obj
 0001:00003462       _AdjustEndianessArray16    10004462 f   cmsio1.obj
 0001:00003477       _Convert15Fixed16          10004477 f   cmsio1.obj
 0001:000034d7       _ReadBase                  100044d7 f   cmsio1.obj
 0001:00003514       _DecodeDateTimeNumber      10004514 f   cmsio1.obj
 0001:000035c1       _EncodeDateTimeNumber      100045c1 f   cmsio1.obj
 0001:00003667       _NormalizeXYZ              10004667 f   cmsio1.obj
 0001:000036ba       _EvalCHRM                  100046ba f   cmsio1.obj
 0001:000036f7       _ReadHeader                100046f7 f   cmsio1.obj
 0001:000039f4       _FixLUT8                   100049f4 f   cmsio1.obj
 0001:00003ae3       _FixLUT8bothSides          10004ae3 f   cmsio1.obj
 0001:00003ba1       _ReadLUT8                  10004ba1 f   cmsio1.obj
 0001:000040f3       _ReadLUT16                 100050f3 f   cmsio1.obj
 0001:00004440       _ReadCurve                 10005440 f   cmsio1.obj
 0001:0000464b       _ReadCurveReversed         1000564b f   cmsio1.obj
 0001:00004883       _ReadMatrixOffset          10005883 f   cmsio1.obj
 0001:00004960       _ReadCLUT                  10005960 f   cmsio1.obj
 0001:00004a89       _ReadSetOfCurves           10005a89 f   cmsio1.obj
 0001:00004bbf       _ReadLUT_A2B               10005bbf f   cmsio1.obj
 0001:00004d20       _ReadLUT_B2A               10005d20 f   cmsio1.obj
 0001:00004f8f       _ReadICCXYZ                10005f8f f   cmsio1.obj
 0001:0000504b       _ReadICCXYZArray           1000604b f   cmsio1.obj
 0001:0000532f       _CheckHeader               1000632f f   cmsio1.obj
 0001:000055ed       _ReadCriticalTags          100065ed f   cmsio1.obj
 0001:00005767       _SaveWordsTable            10006767 f   cmsio1.obj
 0001:000057ab       _SaveHeader                100067ab f   cmsio1.obj
 0001:0000590f       _SetupBase                 1000690f f   cmsio1.obj
 0001:0000593e       _SaveXYZNumber             1000693e f   cmsio1.obj
 0001:000059b7       _SaveXYZArray              100069b7 f   cmsio1.obj
 0001:00005a59       _SaveGammaTable            10006a59 f   cmsio1.obj
 0001:00005aa7       _SaveGammaOneValue         10006aa7 f   cmsio1.obj
 0001:00005b1f       _SaveGammaParametric       10006b1f f   cmsio1.obj
 0001:00005bf1       _SaveGamma                 10006bf1 f   cmsio1.obj
 0001:00005c3d       _SaveDescription           10006c3d f   cmsio1.obj
 0001:00005cc6       _SaveOneChromaticity       10006cc6 f   cmsio1.obj
 0001:00005d32       _SaveChromaticities        10006d32 f   cmsio1.obj
 0001:00005dfc       _SaveSequenceDescriptionTag 10006dfc f   cmsio1.obj
 0001:00005ed1       _SaveDateTimeNumber        10006ed1 f   cmsio1.obj
 0001:00005f0c       _SaveNamedColorList        10006f0c f   cmsio1.obj
 0001:000060d3       _SaveColorantTable         100070d3 f   cmsio1.obj
 0001:000061a3       _SaveLUT                   100071a3 f   cmsio1.obj
 0001:000063a8       _SaveLUT8                  100073a8 f   cmsio1.obj
 0001:0000662d       _SaveTagDirectory          1000762d f   cmsio1.obj
 0001:000066da       _SaveTags                  100076da f   cmsio1.obj
 0001:00006e32       _DupBlockTab               10007e32 f   cmslut.obj
 0001:000079ff       _EvalLUTdoubleKLab         100089ff f   cmslut.obj
 0001:00007a92       _ComputeJacobianLab        10008a92 f   cmslut.obj
 0001:00007d0f       _ComputeTables             10008d0f f   cmsmatsh.obj
 0001:00007dca       _AllSmeltedBehaviour       10008dca f   cmsmatsh.obj
 0001:00007f33       _InputBehaviour            10008f33 f   cmsmatsh.obj
 0001:00008022       _OutputBehaviour           10009022 f   cmsmatsh.obj
 0001:0000847d       _RangeCheck                1000947d f   cmsmtrx.obj
 0001:00008a10       _GrowNamedColorList        10009a10 f   cmsnamed.obj
 0001:00008bbf       _UnrollAnyBytes            10009bbf f   cmspack.obj
 0001:00008bff       _Unroll4Bytes              10009bff f   cmspack.obj
 0001:00008c45       _Unroll4BytesReverse       10009c45 f   cmspack.obj
 0001:00008c9f       _Unroll4BytesSwapFirst     10009c9f f   cmspack.obj
 0001:00008ce5       _Unroll4BytesSwap          10009ce5 f   cmspack.obj
 0001:00008d2b       _Unroll4BytesSwapSwapFirst 10009d2b f   cmspack.obj
 0001:00008d71       _UnrollAnyWords            10009d71 f   cmspack.obj
 0001:00008daa       _Unroll4Words              10009daa f   cmspack.obj
 0001:00008dd7       _Unroll4WordsReverse       10009dd7 f   cmspack.obj
 0001:00008e18       _Unroll4WordsSwapFirst     10009e18 f   cmspack.obj
 0001:00008e45       _Unroll4WordsSwap          10009e45 f   cmspack.obj
 0001:00008e72       _Unroll4WordsSwapSwapFirst 10009e72 f   cmspack.obj
 0001:00008e9f       _Unroll4WordsBigEndian     10009e9f f   cmspack.obj
 0001:00008ee6       _Unroll4WordsBigEndianReverse 10009ee6 f   cmspack.obj
 0001:00008f42       _Unroll4WordsSwapBigEndian 10009f42 f   cmspack.obj
 0001:00008f89       _Unroll3Bytes              10009f89 f   cmspack.obj
 0001:00008fc0       _Unroll3BytesLab           10009fc0 f   cmspack.obj
 0001:00008fe3       _Unroll3BytesSwap          10009fe3 f   cmspack.obj
 0001:0000901a       _Unroll3Words              1000a01a f   cmspack.obj
 0001:0000903e       _Unroll3WordsSwap          1000a03e f   cmspack.obj
 0001:00009062       _Unroll3WordsBigEndian     1000a062 f   cmspack.obj
 0001:0000909a       _Unroll3WordsSwapBigEndian 1000a09a f   cmspack.obj
 0001:000090d2       _Unroll1Byte               1000a0d2 f   cmspack.obj
 0001:000090f3       _Unroll1ByteSkip2          1000a0f3 f   cmspack.obj
 0001:00009114       _Unroll1ByteReversed       1000a114 f   cmspack.obj
 0001:0000913c       _Unroll1Word               1000a13c f   cmspack.obj
 0001:00009156       _Unroll1WordReversed       1000a156 f   cmspack.obj
 0001:00009174       _Unroll1WordBigEndian      1000a174 f   cmspack.obj
 0001:0000919a       _Unroll1WordSkip3          1000a19a f   cmspack.obj
 0001:000091b4       _Unroll2Byte               1000a1b4 f   cmspack.obj
 0001:000091e6       _Unroll2ByteSwapFirst      1000a1e6 f   cmspack.obj
 0001:00009218       _Unroll2Word               1000a218 f   cmspack.obj
 0001:0000923b       _Unroll2WordSwapFirst      1000a23b f   cmspack.obj
 0001:0000925e       _Unroll2WordBigEndian      1000a25e f   cmspack.obj
 0001:00009293       _UnrollPlanarBytes         1000a293 f   cmspack.obj
 0001:000092d1       _UnrollPlanarWords         1000a2d1 f   cmspack.obj
 0001:0000930d       _UnrollPlanarWordsBigEndian 1000a30d f   cmspack.obj
 0001:0000934f       _UnrollLabDouble           1000a34f f   cmspack.obj
 0001:000093c2       _UnrollXYZDouble           1000a3c2 f   cmspack.obj
 0001:0000940e       _UnrollInkDouble           1000a40e f   cmspack.obj
 0001:000094bc       _UnrollDouble              1000a4bc f   cmspack.obj
 0001:0000956a       _UnrollDouble1Chan         1000a56a f   cmspack.obj
 0001:000095c9       _PackNBytesDither          1000a5c9 f   cmspack.obj
 0001:0000961c       _PackNBytesSwapDither      1000a61c f   cmspack.obj
 0001:00009668       _PackNBytes                1000a668 f   cmspack.obj
 0001:000096b1       _PackNBytesSwap            1000a6b1 f   cmspack.obj
 0001:000096f4       _PackNWords                1000a6f4 f   cmspack.obj
 0001:0000972d       _PackNWordsSwap            1000a72d f   cmspack.obj
 0001:00009760       _PackNWordsBigEndian       1000a760 f   cmspack.obj
 0001:000097a1       _PackNWordsSwapBigEndian   1000a7a1 f   cmspack.obj
 0001:000097db       _PackPlanarBytes           1000a7db f   cmspack.obj
 0001:0000981e       _PackPlanarWords           1000a81e f   cmspack.obj
 0001:00009856       _Pack6Bytes                1000a856 f   cmspack.obj
 0001:000098d1       _Pack6BytesSwap            1000a8d1 f   cmspack.obj
 0001:0000994c       _Pack6Words                1000a94c f   cmspack.obj
 0001:0000998f       _Pack6WordsSwap            1000a98f f   cmspack.obj
 0001:000099d2       _Pack6WordsBigEndian       1000a9d2 f   cmspack.obj
 0001:00009a37       _Pack6WordsSwapBigEndian   1000aa37 f   cmspack.obj
 0001:00009a9c       _Pack4Bytes                1000aa9c f   cmspack.obj
 0001:00009af3       _Pack4BytesReverse         1000aaf3 f   cmspack.obj
 0001:00009b60       _Pack4BytesSwapFirst       1000ab60 f   cmspack.obj
 0001:00009bb7       _Pack4BytesSwap            1000abb7 f   cmspack.obj
 0001:00009c0e       _Pack4BytesSwapSwapFirst   1000ac0e f   cmspack.obj
 0001:00009c65       _Pack4Words                1000ac65 f   cmspack.obj
 0001:00009c92       _Pack4WordsReverse         1000ac92 f   cmspack.obj
 0001:00009cd3       _Pack4WordsSwap            1000acd3 f   cmspack.obj
 0001:00009d00       _Pack4WordsBigEndian       1000ad00 f   cmspack.obj
 0001:00009d47       _Pack4WordsBigEndianReverse 1000ad47 f   cmspack.obj
 0001:00009da1       _Pack4WordsSwapBigEndian   1000ada1 f   cmspack.obj
 0001:00009de8       _Pack3Bytes                1000ade8 f   cmspack.obj
 0001:00009e2d       _Pack3BytesLab             1000ae2d f   cmspack.obj
 0001:00009e48       _Pack3BytesSwap            1000ae48 f   cmspack.obj
 0001:00009e8d       _Pack3Words                1000ae8d f   cmspack.obj
 0001:00009eb1       _Pack3WordsSwap            1000aeb1 f   cmspack.obj
 0001:00009ed5       _Pack3WordsBigEndian       1000aed5 f   cmspack.obj
 0001:00009f0d       _Pack3WordsSwapBigEndian   1000af0d f   cmspack.obj
 0001:00009f45       _Pack3BytesAndSkip1        1000af45 f   cmspack.obj
 0001:00009f8c       _Pack3BytesAndSkip1SwapFirst 1000af8c f   cmspack.obj
 0001:00009fd2       _Pack3BytesAndSkip1Swap    1000afd2 f   cmspack.obj
 0001:0000a018       _Pack3BytesAndSkip1SwapSwapFirst 1000b018 f   cmspack.obj
 0001:0000a05f       _Pack3WordsAndSkip1        1000b05f f   cmspack.obj
 0001:0000a083       _Pack3WordsAndSkip1Swap    1000b083 f   cmspack.obj
 0001:0000a0a9       _Pack3WordsAndSkip1SwapSwapFirst 1000b0a9 f   cmspack.obj
 0001:0000a0cd       _Pack3WordsAndSkip1BigEndian 1000b0cd f   cmspack.obj
 0001:0000a105       _Pack3WordsAndSkip1SwapBigEndian 1000b105 f   cmspack.obj
 0001:0000a13f       _Pack1Byte                 1000b13f f   cmspack.obj
 0001:0000a15d       _Pack1ByteAndSkip1         1000b15d f   cmspack.obj
 0001:0000a17d       _Pack1ByteAndSkip1SwapFirst 1000b17d f   cmspack.obj
 0001:0000a19c       _Pack1Word                 1000b19c f   cmspack.obj
 0001:0000a1ae       _Pack1WordBigEndian        1000b1ae f   cmspack.obj
 0001:0000a1c6       _Pack1WordAndSkip1         1000b1c6 f   cmspack.obj
 0001:0000a1d8       _Pack1WordAndSkip1SwapFirst 1000b1d8 f   cmspack.obj
 0001:0000a1ec       _Pack1WordAndSkip1BigEndian 1000b1ec f   cmspack.obj
 0001:0000a204       _PackLabDouble             1000b204 f   cmspack.obj
 0001:0000a271       _PackXYZDouble             1000b271 f   cmspack.obj
 0001:0000a2d1       _PackInkDouble             1000b2d1 f   cmspack.obj
 0001:0000a34b       _PackDouble                1000b34b f   cmspack.obj
 0001:0000ac3f       _CubeRoot                  1000bc3f f   cmspcs.obj
 0001:0000acf7       _f                         1000bcf7 f   cmspcs.obj
 0001:0000ad20       _f_1                       1000bd20 f   cmspcs.obj
 0001:0000b0ed       _Clamp_L_double            1000c0ed f   cmspcs.obj
 0001:0000b118       _Clamp_ab_double           1000c118 f   cmspcs.obj
 0001:0000b2c0       _XYZ2Fix                   1000c2c0 f   cmspcs.obj
 0001:0000b6b9       _XFormSampler              1000c6b9 f   cmssamp.obj
 0001:0000b7bf       _BlackPreservingGrayOnlySampler 1000c7bf f   cmssamp.obj
 0001:0000b821       _BlackPreservingSampler    1000c821 f   cmssamp.obj
 0001:0000b9c4       _EstimateTAC               1000c9c4 f   cmssamp.obj
 0001:0000ba05       _BlackPreservingEstimateErrorSampler 1000ca05 f   cmssamp.obj
 0001:0000bc62       _PatchLUT                  1000cc62 f   cmssamp.obj
 0001:0000c0a5       _Create3x3EmptyLUT         1000d0a5 f   cmsvirt.obj
 0001:0000c413       _ComputeChromaticAdaptation 1000d413 f   cmswtpnt.obj
 0001:0000c66c       _BlackPointAsDarkerColorant 1000d66c f   cmswtpnt.obj
 0001:0000c789       _BlackPointUsingPerceptualBlack 1000d789 f   cmswtpnt.obj
 0001:0000c8c2       _GetV4PerceptualBlack      1000d8c2 f   cmswtpnt.obj
 0001:0000c9be       _ShaperMatrixToPCS         1000d9be f   cmsxform.obj
 0001:0000c9d9       _LUTtoPCS                  1000d9d9 f   cmsxform.obj
 0001:0000c9f4       _NC2toPCS                  1000d9f4 f   cmsxform.obj
 0001:0000ca38       _PCStoShaperMatrix         1000da38 f   cmsxform.obj
 0001:0000ca53       _PCStoLUT                  1000da53 f   cmsxform.obj
 0001:0000ca6e       _NullXFORM                 1000da6e f   cmsxform.obj
 0001:0000cab3       _NormalXFORM               1000dab3 f   cmsxform.obj
 0001:0000cc67       _PrecalculatedXFORM        1000dc67 f   cmsxform.obj
 0001:0000cceb       _TransformOnePixelWithGamutCheck 1000dceb f   cmsxform.obj
 0001:0000cd48       _PrecalculatedXFORMGamutCheck 1000dd48 f   cmsxform.obj
 0001:0000cd9e       _CachedXFORM               1000dd9e f   cmsxform.obj
 0001:0000cee4       _CachedXFORMGamutCheck     1000dee4 f   cmsxform.obj
 0001:0000cff6       _MatrixShaperXFORM         1000dff6 f   cmsxform.obj
 0001:0000d04e       _NC2deviceXform            1000e04e f   cmsxform.obj
 0001:0000d0b6       _FromLstarToXYZ            1000e0b6 f   cmsxform.obj
 0001:0000d1d8       _cmsBuildGrayInputMatrixShaper 1000e1d8 f   cmsxform.obj
 0001:0000d2f0       _cmsBuildGrayOutputMatrixShaper 1000e2f0 f   cmsxform.obj
 0001:0000d58d       _cmsBuildSmeltMatShaper    1000e58d f   cmsxform.obj
 0001:0000d6c9       _GetPhase                  1000e6c9 f   cmsxform.obj
 0001:0000d6f9       _TakeConversionRoutines    1000e6f9 f   cmsxform.obj
 0001:0000d9ff       _IsProperColorSpace        1000e9ff f   cmsxform.obj
 0001:0000da39       _AllocEmptyTransform       1000ea39 f   cmsxform.obj
 0001:0000dacf       _SetPrecalculatedTransform 1000eacf f   cmsxform.obj
 0001:0000db5f       _CreateProof               1000eb5f f   cmsxform.obj
 0001:0000dc7a       _PickTransformRoutine      1000ec7a f   cmsxform.obj
 0001:0000dfa3       _MultiprofileSampler       1000efa3 f   cmsxform.obj
 0001:0000dfe7       _IsAllowedInSingleXform    1000efe7 f   cmsxform.obj
 0001:0000e00a       _CreateDeviceLinkTransform 1000f00a f   cmsxform.obj
 0001:0000e946       _TransportValue32          1000f946 f   LCMS.obj
 0001:0000e946       _TransportValue32          1000f946 f   LCMS.obj
